:100000000828FFFFFFFFFFFFF52BCB2A8A018200A4
:10001000FF308E00FF308F00EA220A306123111278
:10002000AC230330E12232307A230330E122323034
:100030007A230330E12232307A233230D52228303D
:10004000D522AF229322AD220F17CA238F16CB23BE
:100050008F17C9230E11CE238C10BB226030A10054
:10006000CE30A20030302C22E32107220130A00044
:10007000A32321089A000230A000A323210898009E
:100080000330A000A32321089B0018086C3C031C2C
:100090005E280430A000A32321089D000530A000A5
:1000A000A32321089C000630A000A323210894006C
:1000B0000730A000A3232108950062280B309C0084
:1000C00046309D0098218921023061236030A100D3
:1000D000CE30A20000302C22061F7F286030A10005
:1000E000CE30A20010302C229F018B20F7208C10E4
:1000F0006030A100CE30A20000302C2289218C1C5F
:100100007221861E85281015AE23861F892810119E
:10011000AE236C288A281F08033C03199D28061F5C
:1001200094289F0A01305A231F08013C03199E207E
:100130001F08023C0319F7208B28BB2A98211015B1
:10014000AE23B9225330CD226530CD227430CD227A
:100150002030CD224630CD227230CD227130CD22DA
:100160002030CD22861FC72805301D029D001D08A6
:10017000053E9E0005301E020318C12801301C02F6
:100180009C0005301E020318C72864309D07861E98
:10019000D12805309D071D085F3C0318D1289C0A13
:1001A0009D011C08163C031DDC281D08053C031D91
:1001B000DC2801309C009D0101301C020318E3285B
:1001C00016309C009D011C08563E98001808633CA0
:1001D0000318ED2801309A00EE289A011D085F3CB3
:1001E000031C9D011A211D089B0001305A2B013070
:1001F000A0001A0892230230A000180892230330AE
:10020000A0001B0892230430A0001D089223053093
:10021000A0001C0892230630A00014089223073087
:10022000A000150892231A2198210530612303307C
:100230009F0008001D08A9000A30AA00E5232B082A
:10024000A00020089900180892001308A1001208C5
:10025000A2001708A3000A304C21210893002208AD
:100260009200230897009401950112081907940041
:1002700013080318013E170795001708A100150879
:10028000A2001408A30002304C2121089700220884
:100290009500230894000800A4002208A100230868
:1002A000A200A3012108A5002208A6000830A7008B
:1002B000A40C03186029A70B5829A101A20100343E
:1002C00003106B29A40C031C6B292608A207250820
:1002D0000318250FA107A10CA20CA30CA70B6229E0
:1002E000003408006030A10036222208A000201F40
:1002F00088296030A100CE30A20024302C22982121
:100300008C14B9222030CD222030CD22013061233F
:100310000800B9225530CD224E30CD224C30CD22AE
:100320004F30CD224330CD224B30CD220130612BD6
:100330001B08553C0319C0291B085F3C0319C02941
:100340001B084B3C0319C0291B08413C0319C02959
:100350001B08373C0319C0291B082D3C0319C02971
:100360001B08233C0319C0291B08193C0319C02989
:100370001B080F3C0319C0291B08053C031DC42999
:100380001408013E9600C62914089600B7220430CE
:10039000A1001A08A2002030F6220430A10018089B
:1003A000A200303009232E30CD220430A1001B08DA
:1003B000A200303009236030A1001508A200160801
:1003C0002C220130612BB9225030CD224C30CD226D
:1003D0004C30CD222030CD225430CD225230CD228F
:1003E0004130CD224E30CD22B7225330CD224D3078
:1003F000CD224930CD225430CD225430CD2245304B
:10040000CD225230CD222030CD220130532BB922C3
:100410004830CD224A30CD224830CD222730CD225F
:100420005330CD226F30CD226630CD227430CD22B4
:10043000B7222030CD222630CD222030CD2252309E
:10044000CD224430CD225630CD225630CD22203020
:10045000CD2201305323BB2AA30021083D222208CC
:1004600056226622230856226622932AA2002108D9
:1004700043224A222308A200622AA400A0220310D9
:10048000240D5622662AA300A0220310230D013E4C
:100490005622662AA3000830A4000310A30D73227D
:1004A00023100C192314A40B4D2A0800A5000830B2
:1004B000A6000C11A51B0C1584220310A50DA60B7C
:1004C000592A08006422932A0C11842AAD228E1422
:1004D000CF23AD220E14D023AD22051C6D2AAD22F0
:1004E0000E10D023AD2AAD228E14CF23AD220E14D0
:1004F000D023AD22051C7A2AAD220C1185180C15CB
:10050000AD220E10D023AD2AAD228E100C198E1400
:10051000CF23AD220E14D023AD22051C8D2AAD228F
:100520000E10D023AD2AAD228E10CF23AD220E1097
:10053000D023AD220E14D023AD228E14CF23AD2AAA
:10054000AD228E14CF23AD220E14D023AD228E10F7
:10055000CF23AD220E10D023AD2A0C30852B1010E6
:10056000B0230E10D0239010AF238E10CF2BA830C5
:10057000D52A8030D52A0830D5220130D522C8307E
:100580007A230230D522C8307A230630D5220C30A7
:10059000D522C8307A2B0D08A900A9001116AC236A
:1005A000290E0F39E1222908E12AA1001112AC23FA
:1005B000210E0F39E12282307A232108E122823094
:1005C0007A2BAA009015AD232A08B1239011AD23F0
:1005D000FA30852B0030B1231112AC239011AD23DA
:1005E0000030C0230F12CC238E11CD2BA300220884
:1005F000A6000A30A700D7232808A4002408A200D8
:100600002108A6002208A700230834232808A300F5
:100610000800A3002208A6006430A700D7232808FA
:10062000A4002408A2002108A6002208A9000A307C
:10063000AA00E5232B08A8002808A70023083423D4
:100640002808A3002208A6000A30A700D7232808FC
:10065000A5002508A2002108A6002208A70023085B
:1006600034232808A3000800A800A708031D402B76
:10067000A80803193F2B28088D00260A0620522BB4
:100680000A30270203184A2B2708303E8D00260A1D
:100690000620502B0A302702413E8D00260A0620F4
:1006A0003030A8000800A0002008A2006430A30099
:1006B000C830682BA0002008A2006430A3000A30D4
:1006C000682BA1002108A2006430A3000130682B30
:1006D000A400FF30A5002308A7002208A6001730B9
:1006E00025070318702BA60B6F2BA70B6D2BA40BE4
:1006F0006B2B0800A2002208A300A3080319842B77
:100700000A308523A3037D2B0800AB00F430AC0036
:10071000FC30AD002B082C07031C00342D070318F8
:100720008E2B0800A100200889002108880083166C
:10073000081555308900AA308900881488189E2B26
:10074000081183120800A1002008890083160814EC
:1007500083120808A1000800BA2BBD2BBD2BBD2BAE
:10076000BD2BAB002B080F39AC001108F0392C045D
:100770009100BA2B110886000800100885000800B7
:10078000920012080F3993000F08F03913048F00FC
:10079000D12BD12BD12BD12BD12BD42BD42BD42B70
:1007A000D42B0F08660008000E0865000800A70893
:1007B0000319E22B27082602031CE22B2708260236
:1007C000A600DA2B2608A8000800AC01AA08031925
:1007D000F22B2A082902031CF22B2A082902A9005D
:1007E000AC0AE92B2C08AB00080004308D0008008F
:10400000FFFFFFFFFFFFFFFFFFFFFFFFFFFFFF3F80
:10420000FF00FF00FF00FF00FF00FF00FF00FF00B6
:10421000FF00FF00FF00FF00FF00FF00FF00FF00A6
:10422000FF00FF00FF00FF00FF00FF00FF00FF0096
:10423000FF00FF00FF00FF00FF00FF00FF00FF0086
:10424000FF00FF00FF00FF00FF00FF00FF00FF0076
:10425000FF00FF00FF00FF00FF00FF00FF00FF0066
:10426000FF00FF00FF00FF00FF00FF00FF00FF0056
:10427000FF00FF00FF00FF00FF00FF00FF00FF0046
:00000001FF
